:020000040040BA
:1000000038110020D9064000D5064000D506400032
:10001000D5064000D5064000D5064000000000008F
:10002000000000000000000000000000D5064000B5
:10003000D506400000000000D5064000FD1140003C
:10004000D5064000D5064000D5064000D506400044
:10005000D5064000D5064000D5064000D506400034
:10006000D5064000D506400000000000D50640003F
:10007000D5064000D5064000D5064000D506400014
:10008000D5064000D5064000D5064000D506400004
:10009000AD1B4000D5064000D5064000D506400007
:1000A000D5064000D5064000D5064000D5064000E4
:1000B000D5064000D506400000000000000000000A
:1000C0000000000000000000000000000000000030
:1000D0000000000000000000000000000000000020
:1000E0000000000000000000000000000000000010
:1000F000000000000000000000000000D5064000E5
:10010000ED114000D5064000000000000000000096
:1001100000000000000000000000000000000000DF
:1001200000000000000000000000000000000000CF
:1001300000000000000000000000000000000000BF
:1001400000000000000000000000000000000000AF
:10040000A03F000010B5054C237833B9044B13B15D
:100410000448AFF300800123237010BD00040020C6
:10042000000000009C3D40000C4B43B10C480D49BE
:1004300010B5AFF300800C48036823B910BD0A481B
:10044000036833B97047094B002BF7D0BDE8104063
:100450001847064B002BF5D0184700BF00000000DE
:100460009C3D4000040400209C3D40000000000032
:10047000144B98420FD9144B984211D9134B984200
:1004800012D9134B984213D9124B984214D9124ADD
:10049000124B1A6070474FF08062104B1A60704721
:1004A0000F4A0E4B1A6070470E4A0C4B1A60704789
:1004B0000D4A0A4B1A6070474FF00422074B1A602E
:1004C000704700BF7F9FD500FF3EAB017FDE8002FB
:1004D000FF7D56037F1D2C0400050004000A0E401A
:1004E00000010004000200040003000410B5A0B0E5
:1004F000334A344B1A60344A936843F0254343F43B
:1005000080139360536913F0800F0CD12F4A2E4B48
:100510001A602D4B5B6913F0800FFAD02C4B9B6E49
:1005200013F0800FF5D00023012262F3070343F498
:100530007C53274A936240F6B73161F31C439362C0
:10054000234B9B6E13F0020FFAD00023012262F3BB
:10055000070343F47C531E4AD3624FF4B76161F33F
:100560001A43D3621A4B9B6E13F0040FFAD0022287
:10057000174B1A63164B9B6E13F0080FFAD0154CED
:1005800015482060154B98472268154B1344154AAF
:10059000934201D920B010BD20216846124B9847E4
:1005A0000949CB6923F4F053109A520202F4F05235
:1005B000134343F0B44343F48073CB61EAE700BFD5
:1005C00000050004000A0E4010140E40080000A5AB
:1005D00000040E40B80900200000DC057104400052
:1005E000C0D3BDF980C3C9010D00002010B50C4B6C
:1005F0009847044601220B4B9A600A4B1B6913F083
:10060000010F0AD0064B984704F114039842F4D91D
:100610000122044BDA60002010BD012010BD00BF94
:100620002D1640000080044010B400240EE040006D
:1006300080F00700C0B20133DBB2072B05D810F001
:10064000800FF4D14000C0B2F5E70134944204D2E7
:1006500011F8013B58400023EFE710BC7047000041
:1006600070B506460D464FF40032164BC3F8002114
:100670000122154B5A63154B00241C605C609C6082
:10068000DC601C610AE0114A53602C460E4B0F4A95
:100690001A6001229A630E4B984788B1AC420CD283
:1006A000A3190A4A13602B1B4FF6F8729342EAD93A
:1006B0001346064A53601C44E8E7034BD86B70BDF1
:1006C000002070BD00040E4000800440000A00209D
:1006D000ED054000FEE7000008B5104B104A9A42B5
:1006E00009D00E4B0E4A03E011681960043304323E
:1006F0000C498B42F8D30C4B02E000221A60043301
:100700000A4A9342F9D30A4A0A4B23F07F039360C3
:10071000094B9847094B9847FEE700BF0C000020A3
:100720009C3D40000402002000040020340B002007
:1007300000ED00E000004000413C40008D1A400008
:10074000014A024B1A60704700127A0090010020A3
:10075000A0F58000012915D0430A19B1022918D04B
:1007600002207047430B1B0323F07F430E481843BE
:1007700010B5EFF3108404B972B60C4B984794B9D6
:1007800062B610BD830B5B0323F07F430848184318
:10079000EEE7180220F07F4020F0FF0040F0B44068
:1007A00040F01100E4E710BD0702005A710000207C
:1007B0000703005A38B502210A480B4B98470546F3
:1007C00068B90124032C0AD804F120000221400456
:1007D000054B984710B90134E4B2F3E705462846C3
:1007E00038BD00BF00404000510740002DE9F041F6
:1007F00006460C461546EFF3108707B972B6A6F504
:100800008000400A1FFA80FE0EF5005E4FEA4E2E71
:10081000A6EB0E0806EB040CAEEB0C0101F5007123
:10082000002305E04FF0FF324EF8232001339BB246
:10083000B3EB980FF6D3B646002305E055F8232016
:100840004EF8232001339BB2B3EB940FF6D3E64668
:10085000002305E04FF0FF324EF8232001339BB216
:10086000B3EB910FF6D3000220F07F4020F0FF00A1
:1008700040F0B44040F001000E4B9847864670B1FE
:10088000AFB962B613E004339BB29C420AD99A080E
:1008900055F82210F2589142F5D00130F3E70020CC
:1008A0000346F2E707B962B608B14FF0030E70468F
:1008B000BDE8F0817100002010B5EFF3108404B999
:1008C00072B60348034B984704B962B610BD00BF27
:1008D0001300005A7100002010B5EFF3108404B922
:1008E00072B6002307E09A0002F5800250F8231048
:1008F000116001339BB27F2BF5D90348034B984716
:1009000004B962B610BD00BF1200005A7100002089
:1009100038B50246EFF3108404B972B68023034958
:100920000348044DA84704B962B638BD1500005A03
:100930001400005AFD000020154B98421BD003F50F
:10094000A033984219D003F58043984217D0A3F5FD
:100950004043984215D003F58043984213D0A3F545
:10096000A033984211D003F56033984201D0322071
:1009700070471620704708207047092070470E20E6
:10098000704713207047142070471520704700BF30
:1009900000C0004031281BD81F280BD80D4B9A6986
:1009A00001238340934313D0012303FA00F0094B42
:1009B000186170472038074BD3F808210123834082
:1009C000934305D0012303FA00F0024BC3F8000162
:1009D000704700BF00040E404900B0FBF1F003383F
:1009E000002302E040080133DBB2FF28FAD80202FC
:1009F00002F47F4252FA80F01B0403F4E02318440F
:100A000070470368027AD2B2012A21D010B403F5EC
:100A1000C063012202720022C271C1604A78012AB9
:100A200012D00A78120402F4FE025A608C68C2796D
:100A3000D2B2511CC9B2C171A25C5A634FF4417267
:100A40005A62012010BC70470A7852081204ECE781
:100A5000002070470268037ADBB2012B27D010B464
:100A600002F5C064012303720023C371C1604B7897
:100A7000012B12D00B781B0403F4FE0303F5805303
:100A800063600B79012B0ED00123C2F8003640F2CF
:100A900002336362012010BC70470B785B081B04B3
:100AA00003F58053ECE70323C2F80036EFE700209C
:100AB0007047036803F5C063027AD2B2012A17D0E7
:100AC000012202720022C271C1604A78012A0BD051
:100AD0000A78120402F4FE025A60CA785A634FF48C
:100AE00041725A62012070470A7852081204F3E7F3
:100AF00000207047036803F5C063027AD2B2012A6E
:100B000017D0012202720022C271C1604A78012A04
:100B10000BD00A78120402F4FE025A60CA785A63B3
:100B20004FF441725A62012070470A785208120449
:100B3000F3E70020704782B00023ADF8063006E0EE
:100B4000BDF806309BB201339BB2ADF80630BDF85C
:100B500006309BB2B3F52F7FF2D302B0704700008E
:100B60002DE9F04106468846046820461B4B98470D
:100B7000312801D9BDE8F0810546194B9847032378
:100B800023608023C4F800362423C4F8003641468D
:100B90001448154B9847C4F81006002333720123FC
:100BA000B3716BB2002B07DB5A0905F01F0001215E
:100BB00081400E4840F82210002B08DB03F160430F
:100BC00003F56143202283F80023BDE8F08105F09E
:100BD0000F05074B20225A55CCE700BF39094000CA
:100BE000950940000000DC05D909400000E100E063
:100BF00014ED00E008B5837993B18B78032B11D8FD
:100C0000DFE803F00205080B074B984708BD074BC8
:100C1000984708BD064B984708BD064B984708BD46
:100C2000002008BD002008BD030A4000550A40000E
:100C3000B30A4000F50A4000007A7047F8B506464E
:100C4000036803F5C064256AC76815F0040F0BD06C
:100C5000E26A12F0040F07D0BA78002A4DD0022AB7
:100C60004BD0BA78032A5ED015F0020F08D0E26AA2
:100C700012F0020F04D0BA78012A73D0032A71D07F
:100C800015F4807F0DD0E36A13F4807F09D040F221
:100C90000733A362002333720323B371FB6803B1EC
:100CA000984715F4007F0DD0E36A13F4007F09D054
:100CB00040F20733A362002333720423B371FB684D
:100CC00003B1984715F0010F16D0E36A13F0010F36
:100CD00012D0BB780BB1022B09D140F20533A362CD
:100CE000002333720223B371FB6803B19847BB78CA
:100CF000012B54D0032B52D0F8BDF279D2B23979FE
:100D00008A4208D2B868F279D2B2511CC9B2F171E4
:100D1000825C6263A5E70222C3F8002601226262B8
:100D20000422A2629DE77A78012A11D03A7812044F
:100D300002F4FE0202F5805262603A79012A0DD077
:100D40000122C3F800260422A262022262628BE71B
:100D50003A785208120402F58052EDE70322C3F8F4
:100D60000026F0E7B868F279D2B2511CC9B2F1712D
:100D7000216B8154F179C9B23A79013A91420AD092
:100D8000F379DBB23A7993427FF47AAF012363625D
:100D90000223A36274E70222C3F80026F0E740F2C0
:100DA0000333A362002333720223B371FB68002B69
:100DB000A2D09847A0E70000F8B50379202B0BD903
:100DC000A3F12006F3B20B4F01269E403E603E6524
:100DD0003E613E63002408E0074FF5E7074DA84752
:100DE0007E63A8473E630134E4B2092CF6D97E61E4
:100DF0007E60F8BD00100E40000E0E40370B400024
:100E0000014B1868704700BF0044400008B5024B12
:100E10009847024B185808BD010E400000404000A2
:100E200008B5044B984701460348044B9847C04314
:100E300008BD00BF010E40000040400061064000B8
:100E4000F8B5036841681B4A9A4227D81A4D1B4AD5
:100E50009A4225D91A4B8B4224D88D4224D9044674
:100E6000184B98470027061947F10007012F08BFC4
:100E7000002E1BD2B0F5847F1AD30023BB4208BFDB
:100E8000B54201D20020F8BD0F4B984704460F4BE6
:100E90009847844214BF00200120F8BD0020F8BD0F
:100EA0000020F8BD0020F8BD0020F8BD0020F8BDEE
:100EB0000020F8BD00000020000048000080022053
:100EC00000004000010E4000210E40000D0E4000C9
:100ED0002DE9F8430378442B02D00220BDE8F883C3
:100EE0004578A5F10803DBB2182B02D90520BDE82F
:100EF000F88315F0070F02D00520BDE8F883867847
:100F0000C37806EB0326037906EB0346437906EB29
:100F100003661E4A1E4B9E4202D20420BDE8F8839F
:100F2000964202D30420BDE8F8835FFA85F84FF0BB
:100F3000000918EB060849F10009B9F1010F08BFD3
:100F4000B8F1000F02D30420BDE8F88300234B451D
:100F500008BF424502D20420BDE8F8830446AA1D1A
:100F6000875C014600200B4B9847874202D0062041
:100F7000BDE8F88306F4FE762A46A11D06483044F3
:100F8000064B98470020BDE8F88300BF00004800EA
:100F900000404000290640001C040020893C40001D
:100FA000F8B50378642B01D00220F8BD4678A6F18D
:100FB0000803DBB2182B01D90520F8BD8578C3786A
:100FC00005EB0325037905EB0345437905EB036541
:100FD000B5F5007F01D30420F8BDF2B20023521909
:100FE00043F10003012B08BF002A01D30420F8BD00
:100FF000AB19B3F5007F01D90420F8BD0446B21D3A
:10100000875C01460020084B9847874201D00620A4
:10101000F8BDC5F38F053246A11D044800EB8500DD
:10102000034B98470020F8BD290640001C0600200D
:10103000893C40000378652B01D00220704770B5D1
:101040008478C37804EB0324037904EB03444379E5
:1010500004EB0364214B9C4201D3042070BD204B60
:101060009C4201D2042070BD4378012B14D01BB1E7
:10107000022B18D0022070BDC4F30C030BB1042066
:1010800070BD00260146857906220020154B984741
:1010900085421ED0062070BDC4F30D030BB10420A1
:1010A00070BD0126EEE7104B9C420CD0B4F5840FC6
:1010B0000BD0B4F5880F0AD0B4F58C0F01D0042002
:1010C00070BD0226DEE70226DCE70226DAE702260A
:1010D000D8E731462046054B984770BD00004800D0
:1010E00000404000290640000040400051074000F9
:1010F0002DE9F8430378502B03D002242046BDE8A5
:10110000F88343780BB10524F8E78478C27804EBC0
:101110000224027904EB0244427904EB02641D4E7E
:101120001D4A944201D20424E8E7B44201D30424C6
:10113000E4E75FFA83F84FF0000918EB040849F17F
:101140000009B9F1010F08BFB8F1000F01D3042461
:10115000D4E700274F4508BF464501D20424CDE718
:1011600001469A1D855C00200C4B9847854201D0B2
:101170000624C3E70A4D2A464FF400712046094B66
:10118000984704464FF40072FF212846064B9847C3
:10119000B4E700BF000048000040400029064000BE
:1011A0001C040020ED0740009F3C400038B5037848
:1011B000702B02D00224204638BD084B98470446C5
:1011C0000028F8D1064D2846064B984704464FF4B0
:1011D0000072FF212846044B9847ECE7B90840000D
:1011E0001C060020D90840009F3C400008B50020A4
:1011F000014B984708BD00BFE9374000034AD2F8C9
:1012000000340133C2F80034704700BF1C040020D2
:10121000044B01229A6380221A604FF48032C3F893
:101220000021704700040E404FF4C052134B1A6166
:10123000134AD2F8143123F44063C2F81431D2F8BF
:10124000203143F00103C2F820310E4B4FF44061CE
:101250005960196F21F440611967D2F8141141F0F7
:101260002001C2F814114FF400721A601A615A6317
:1012700020221A601A615A63704700BF00040E40B2
:1012800000020E4000100E4000207047F8B51C46CA
:10129000BDF818501B78223B4E2B00F26D81DFE821
:1012A00013F073006B016B016B016B016B016B0140
:1012B0006B014F006B016B016B016B016B016B01EB
:1012C0006B016B016B016B016B016B016B016B01BE
:1012D0006B016B016B016B016B016B016B016B01AE
:1012E0006B016500C9009C006B016B016B016B0118
:1012F00061016B016B016B01E1006B016B01B400DB
:101300006B016B012A016B016B016B016B016B01BE
:101310006B016B016B016B016B016B016B016B016D
:101320006B016B016B01000187006B016B016B01AD
:101330006B016B016B016B016B016B016B011501A3
:10134000964C04F204462A4600213046944B9847B6
:10135000944B93E80300C4F8040484F80814EBB237
:10136000324600210846904CA047F8BD8F4A93684A
:1013700023F07F4323F4706343F0254343F4E06399
:1013800093608B4B1360F8BD8A4B98470746834E9A
:1013900006F204442A4600212046814B984786F8ED
:1013A0000474EBB22246002108467F4CA047F8BDEA
:1013B0002046814B98470746784E06F204442A4659
:1013C00000212046764B984786F80474EBB22246FB
:1013D00000210846744CA047F8BD2046774B98473B
:1013E0000446002800F0D8806C4F07F204462A46D5
:1013F000002130466A4B984787F80444EBB23246E6
:1014000000210846684CA047F8BD20466C4B984721
:101410000746624E06F204442A4600212046604BED
:10142000984786F80474EBB22246002108465E4CC9
:10143000A047F8BD634B9847584A82F80704C0F3A9
:10144000072382F80634C0F3074382F80534000E00
:1014500082F80404EBB202F2044200210846524C26
:10146000A047F8BD584B984704464C4E06F2044737
:101470002A46002138464A4B984786F80744C4F369
:10148000072386F80634C4F3074386F80534240E90
:1014900086F80444EBB23A4600210846424CA04785
:1014A000F8BD2046494B984707463C4E06F2044497
:1014B0002A46002120463A4B984786F80474EBB23E
:1014C000224600210846384CA047F8BD2046404B34
:1014D00098470746314E06F204442A46002120462A
:1014E0002F4B984786F80474EBB222460021084639
:1014F0002D4CA047F8BD3748374B9847074680B179
:10150000264E06F204442A4600212046244B9847E2
:1015100086F80474EBB2224600210846224CA0470C
:10152000F8BD1E4F4FF0000E87F804E407F5007475
:101530000FCCC7F80504C7F80914C7F80D24C7F87D
:1015400011340FCCC7F81504C7F81914C7F81D24B7
:10155000C7F82134EBB207F2044271467046124CD0
:10156000A047F8BD1D4BAA221A6042F601425A60FC
:101570000F4A903B1A60F8BD084E2A46002106F239
:101580000440074B9847022386F80434EBB2224606
:1015900000210846044CA047F8BD00BF1C040020F1
:1015A0009F3C4000C03C4000C11B400000140E4066
:1015B000080000A5B507400035104000D10E4000DE
:1015C000F11040000D0E4000210E4000A10F400020
:1015D000AD1140001C0600201109400090140E407F
:1015E00030B587B0044658238DF8083000230593A2
:1015F00001AB049302258DF80C5001238DF80930BE
:101600008DF80A508DF80B108DF804308DF80520F8
:1016100002A9044B98472046034B98470028FAD16B
:1016200007B030BDF50B4000390C4000014BD3F83A
:10163000000470471C04002030B583B00446064DFA
:10164000A8470190A84701E0034B9847019B23441A
:101650009842F9D303B030BD2D164000F0B587B0E5
:1016600000258DF8075010238DF808301C4C1D4BB9
:1016700023602B2323712A2363711B4920461B4BB4
:10168000984720461A4B98471A4F4FF400733B6314
:101690000A20194EB04720233B630A20B047059526
:1016A000E7238DF80B300DF10703049301238DF828
:1016B0000C308DF8093003238DF80A3002A920463A
:1016C0000E4B984706480E4B984703460028F9D121
:1016D000034A9279D2B2022A14D0184607B0F0BD5C
:1016E000180A002000C00140A0860100610B4000E4
:1016F000B90D400000100E4039164000F50B4000B7
:10170000390C40009DF8073043F001038DF8073095
:1017100002238DF80A3002A99048914B98478F48D0
:10172000904B98470028FAD112238DF808300323F4
:101730008DF80A3002A98948894B98478748894B18
:1017400098470028FAD19DF8073043F001038DF83F
:10175000073002238DF80A3002A98048804B984751
:101760007E48804B98470028FAD110238DF8083026
:1017700006238DF80B3003238DF80A3002A9774831
:10178000774B98477548774B98470028FAD19DF8D2
:10179000073063F07F038DF8073002238DF80A309D
:1017A00002A96E486E4B98476C486E4B98470028CC
:1017B000FAD100238DF807300C238DF80B3002A9E5
:1017C0006648674B98476548664B98470028FAD1AA
:1017D0000D238DF80B3002A96048614B98475F4894
:1017E000604B98470028FAD10E238DF80B3002A9E0
:1017F0005A485B4B984759485A4B98470028FAD1AA
:101800000F238DF80B3002A95448554B9847534885
:10181000544B98470028FAD112238DF8083006233C
:101820008DF80B3003238DF80A3002A94B484C4B3E
:1018300098474A484B4B98470028FAD19DF8073003
:1018400063F07F038DF8073002238DF80A3002A978
:101850004248434B98474148424B98470028FAD1A9
:1018600000238DF807300C238DF80B3002A93B487C
:101870003B4B984739483B4B98470028FAD10D23FA
:101880008DF80B3002A93548354B98473348354B16
:1018900098470028FAD10E238DF80B3002A92F4863
:1018A0002F4B98472D482F4B98470028FAD10F23EC
:1018B0008DF80B3002A92948294B98472748294B16
:1018C00098470028FAD110238DF80830E7238DF8C7
:1018D0000B3003238DF80A3002A92048204B98478B
:1018E0001E48204B98470028FAD19DF8073023F076
:1018F00001038DF8073002238DF80A3002A917483A
:10190000174B98471548174B98470028FAD11223D0
:101910008DF80830E7238DF80B3003238DF80A305B
:1019200002A90E480E4B98470C480E4B98470028CA
:10193000FAD19DF8073023F001038DF80730022318
:101940008DF80A3002A90548054B98470348054B16
:1019500098470028FAD10123BFE600BF180A0020EB
:10196000F50B4000390C4000F8B5254C25492046C0
:10197000254B9847254E202777630A20244DA847FA
:101980002046244B98470A20A84737630A20A847D7
:10199000962206212046204B9847A379DBB2022BE2
:1019A00001D00020F8BD25460822072120461A4C08
:1019B000A0477C2209212846A04780220A212846E8
:1019C000A04780220B212846A04700220C21284650
:1019D000A04700220D212846A04700220E212846BC
:1019E000A04700220F212846A0470222F6212846C0
:1019F000A0470122FF212846A0470120F8BD00BFD3
:101A0000180A0020A0860100610B400000100E4063
:101A100039164000B90D4000E115400010B5BFF384
:101A20005F8FBFF36F8F72B600230CE0134A03F190
:101A300020044FF0FF3142F8241003F1600442F813
:101A400024100133DBB2072BF0D900220C4B1A60B3
:101A50004FF480720B4B5A67BFF34F8FBFF36F8FFA
:101A600020F07F02084B9A604368BFF35F8FBFF39B
:101A70006F8F026882F30888984710BD00E100E08C
:101A800010E000E00040044000ED00E010B54FF42D
:101A90000042314B5A6072B6304B9847304B9847F2
:101AA000304B1B68AA2B30D02F4C20462F4B984729
:101AB00058B12C4B1B68BB2B42D12A4B5B681A2BAD
:101AC0003ED1284B00221A605A604FF40072FF2169
:101AD0002748284B9847284B9847284B284A5A6054
:101AE000F021284A82F8231000229A6007221A6007
:101AF000254B9847BFF35F8F62B6244B984738B3A6
:101B0000234B9847234B9847FCE7164B5B6803F43D
:101B10003053B3F5305FC7D1124B5B68DAB2082A95
:101B200007D9104B00221A605A601B4A1B4B1A60DF
:101B3000BAE742F6014252FA83F30A4A5360F4E7E5
:101B4000174B1B68002BC0D02046164B9847BCE7AC
:101B5000154B9847D4E700BF50140E404107400092
:101B6000ED04400090140E4000404000410E400043
:101B70001C0400209F3C40002912400010E000E0BF
:101B8000FF7F010000ED00E0111240005D164000F3
:101B9000B93A4000852F4000080000A500140E400F
:101BA000940100201D1A40006919400008B5024840
:101BB000024B984708BD00BF180A00203D0C4000AA
:101BC000F8B505460F4616461C468C231C4A03FBF7
:101BD0000023597800201B4B9847034600B30FB3EE
:101BE0003F2C28BF3F2416488C2303FB05F3C21863
:101BF000177208331844224631460130124B984779
:101C00000134E4B20E4A8C2000FB05F000F108011B
:101C1000104423460A44417800200C4CA047034658
:101C20001846F8BD402C28BF40248C2303FB05F345
:101C300008332246314602481844034B9847E1E7EF
:101C400060080020C1294000893C4000192A40005A
:101C500008B58C2200210248024B984708BD00BFFE
:101C6000600800209F3C400008B50020014B9847C9
:101C700008BD00BF511C40004B79032B01D0002050
:101C800070472DE9F04182B00B79C3EBC305ADB2CB
:101C90001235ADB295420DD93A4B1B6813F0010FC6
:101CA00064D000BE002002B0BDE8F0818C2202FBAF
:101CB00006460DE0002353B91E468C22324C02FB2F
:101CC00003425278002AF1D00133DBB2F3E7002659
:101CD00076B10B78CC18C6F888406278212A0FD0EC
:101CE000284B1B6813F0010F44D000BE0020DAE738
:101CF000244B1B6813F0010F3AD000BE0020D2E73E
:101D00000F468046C95C3A79731C0193B31C00935B
:101D1000032321441D4CA04730B91A4B1B6813F014
:101D2000010F29D000BEBEE7BB79012B0CD00123E7
:101D30003371BB783370D6F88830B3F80730F3804E
:101D4000B17821B92846AEE7FB79F370EFE740237D
:101D500006F1480240460E4CA04778B9094B1B6873
:101D600013F0010F0CD000BE28469CE700209AE734
:101D7000002098E7002096E7002094E7284692E7A5
:101D8000284690E7F0ED00E0600800203D29400083
:101D9000192A40002DE9F04182B0137803F01F04A6
:101DA000012C04D00023184602B0BDE8F0819488CD
:101DB000E5B20024ACB1FF24002C40F00A811546A6
:101DC0000646274613F0600339D1002940F003810D
:101DD00053881B0A5278062A0DD0062A1CD00023ED
:101DE000E1E78C2606FB04F6824FBE5DB542E3D0E8
:101DF0000134E4B2DEE7212BEFD18C237D4A03FBD3
:101E00000427D7F88820002A00F0E78013782946B5
:101E1000794CA0470346C6E7222B01D00023C2E736
:101E20002046764B98478C23724A03FB0727FB8892
:101E3000024629463046704CA0470123B3E7202BC9
:101E400001D00023AFE75378013B0A2B00F2C78093
:101E5000DFE803F0068C9AC5C5C5C5C54275A80064
:101E6000002940F0BE806B881A0ADFF888C18C20F8
:101E700000FB04F008300CEB0008B5F806E013F0A6
:101E8000FF010CD0BEF1010F1CD908F101030CF8C1
:101E900000100EF1FF3E1FFA8EFE012701E04346BF
:101EA0000027CDF800E02046554CA0473B189BB2D8
:101EB0005BB9544B1B6813F0010F00F0948000BE17
:101EC000002370E743460027EBE7424629463046A9
:101ED000494CA047012366E779B9EB88402B01D92B
:101EE000002360E78C2202FB04F2483241490A4495
:101EF0002946414CA047012355E7022901D001237F
:101F000051E769880A0ADFF8ECE08C2606FB04F644
:101F100048360EEB0603E88811F0FF0105D00128D2
:101F200003D91EF80650A94205D000902046364C31
:101F3000A047012337E70133013880B2F5E70029D4
:101F400053D16988090A8C232A4A03FB0427797133
:101F50002E4B2BB120469847034600283FF423AF71
:101F6000294630462A4B984701231CE709B1012333
:101F700019E78C221F4B02FB04320123053229464C
:101F80001D4CA04701230EE709B101230BE78C226A
:101F9000184B02FB0432012304322946164CA04799
:101FA000012300E719B1022906D00123FBE62946E7
:101FB000174B98470123F6E66988C9B28C220D4B6E
:101FC00002FB04373971134B8BB12046984701232C
:101FD000E9E60023E7E60123E5E60023E3E6002344
:101FE000E1E60123DFE60023DDE60123DBE6012352
:101FF000D9E600BF600800207D324000D53B40009C
:1020000089124000F0ED00E08D1240000000000059
:102010003D32400000000000F0B583B0254D0024A3
:1020200044B1A4B1244B1B6813F0010F3ED000BE95
:10203000002314E08C251F4A05FB0425AA788A4258
:10204000EFD06A789142ECD00134E4B2E8E706467A
:102050006A78914206D0AA7891420DD001231846A1
:1020600003B0F0BD154A1AB3DAB205F108012046F3
:10207000124B98470123F2E705F148079BB2009302
:102080003B460022114620460D4CA04740233A46CD
:10209000A97830460B4CA04703460028DFD1064AFA
:1020A000126812F0010FDAD000BED8E70023D6E79D
:1020B0000123D4E760080020F0ED00E000000000FC
:1020C0008D124000192A40000A4492B2914202D86F
:1020D00083899A4202D94089024492B210467047DD
:1020E0008A1A92B2914202D383899A4202D94089D4
:1020F000121A92B210467047838801E0C91A89B259
:102100008B42FBD908467047F8B504460F46114686
:102110001D46D31A9BB2AA4202D242899B1A9BB295
:10212000A6889E4205D2324620460A4B9847208216
:1021300033460BB90020F8BD29462046064B984788
:102140002168E3881A4603FB00113846034B984781
:102150000120F8BDE1204000F9204000893C40000A
:1021600038B50446C289038A9BB292B2054DA8478E
:102170000546218A82B289B22046034B98472082C5
:10218000284638BD09214000C9204000F8B5C5895E
:10219000ADB2028A92B2AB1A9BB2954202D2428988
:1021A0009B1A9BB282889A4215D00E460446294655
:1021B0000B4B98472768E3881A46314603FB0070AB
:1021C000084B9847012229462046074B9847E08153
:1021D00001231846F8BD037A002BE6D1F9E700BFCA
:1021E000F9204000893C4000C92040000023C38101
:1021F000038283885B009BB2013B9BB28381DB43FC
:10220000438101207047000038B5054600240CE0EA
:10221000E31ADBB2DBB903EB4303DA00194B1344D7
:102220005B68284698470134E4B2174B1B795A1C67
:1022300094420EDA154A42B19C42E9D204EB4403BF
:10224000DA00114B1B681344EAE72346E2E7002358
:10225000E6E70D4C2B22002104F108000C4B9847B7
:102260004FF0FF33C4F80B30C4F80F30C4F813300C
:10227000C4F81730C4F81B30C4F81F30C4F823303A
:1022800038BD00BFC83C4000EC0800200000000042
:102290009F3C400008B5024B9847024B984708BD49
:1022A000092240001533400070B505460C4616461D
:1022B000C868044B9847E36832460021284698478F
:1022C00070BD00BF293340002DE9F84F8046013929
:1022D000C8B26E4B984718B182464378022B09D09A
:1022E0006B4B1B6813F0010F00F0BB8000BE002099
:1022F000BDE8F88FC279C2F3401066490B7A60F3EB
:102300000413C2F3801262F345130B720AF109053C
:10231000BAF802309A447DE02B78A9461D4481E04A
:102320005B4B1B6813F0010F00F09E8000BE002085
:10233000BDE8F88F564B1B6813F0010F00F0978033
:1023400000BE0020BDE8F88FE31ADBB203BB03EB4D
:102350004303514A02EBC3039B6832462946404679
:1023600098478346B0B90134E4B22746494B1B79FC
:102370005A1C944249DA494A42B19C42E4D204EBE5
:102380004403444A126802EBC303E5E72346DDE752
:102390000023E1E7082814D9864212D3AA783D4BDE
:1023A0001344DC72B9F1000F28D099F80220AB7801
:1023B0009A420FD199F804206B799A420AD10123ED
:1023C00018E0334B1B6813F0010F53D000BE002000
:1023D000BDE8F88F2E4B1B6813F0010F4DD000BEE7
:1023E0000020BDE8F88FAA7899182A4A0A44D472C6
:1023F0000133DBB299F803209342F4D323465A46C3
:1024000029462748274CA0475D44224B1B790133BE
:102410009F4217DA55451ED26B780B2B3FF47CAFE9
:102420004FF000096B78042B7FF47AAFAAEB050616
:10243000B6B2AA78174B1344DB7AFF2B7FF47AAF3E
:10244000002492E7124B1B6813F0010F18D000BE56
:102450000020BDE8F88F144BABB198470120BDE8D0
:10246000F88F0020BDE8F88F0020BDE8F88F00202D
:10247000BDE8F88F0020BDE8F88F0020BDE8F88F98
:102480000020BDE8F88F0120BDE8F88FDD3B40005B
:10249000F0ED00E0EC080020C83C40000000000027
:1024A00007090020A13B40000000000038B50546A8
:1024B0000C464888020AC0B2531E0E2B4BD8DFE8E8
:1024C00003F0081C344A4A3F1C4A4A4A4A4A4A4ACC
:1024D0001100284B98471223024621462846264CD5
:1024E000A04738BD254B002B37D09847024643887C
:1024F00021462846204CA04738BD022A0BD0204B4D
:10250000002B2CD0984748B14388024621462846E4
:10251000194CA04738BD1B4B9847F4E71A4B1B6872
:1025200013F0010F1DD000BE38BDA188174B98478E
:102530000246C0B10378214628460F4CA04738BD5B
:10254000134B93B19847024688B103782146284639
:10255000094CA04738BD002038BD002038BD002000
:1025600038BD002038BD002038BD002038BD002017
:1025700038BD00BFCD3B40007D3240000000000070
:1025800000000000DD3B4000F0ED00E0E53B4000D6
:1025900000000000014B93F833007047EC08002066
:1025A000234B93F833300BB11846704770B505468E
:1025B0001F4C2B22002104F108001E4B98471E4E91
:1025C000301D1E4B984766631D4B13B1201D984765
:1025D000206000240FE0E31ADBB23BB903EB4303B6
:1025E000DA00184B134402E02346F6E700231B6889
:1025F00098470134E4B20E4B1B795A1C94420BDA13
:102600000F4A002AF0D09C42E5D204EB4403DA00E2
:10261000074B1B681344EAE728460B4B98472846AC
:102620000A4B98470123024A82F83330184670BD9E
:10263000EC0800209F3C4000DC010020ED21400020
:1026400000000000C83C4000993540006135400062
:1026500070B584B004460D464378023B032B00F26C
:10266000B880DFE803F002832F5A6B4B1A7A6FF3BE
:1026700000021A721A7A6FF341021A72002159721B
:102680001A7A61F382021A725E6B15B93378012BE4
:1026900010D02146301D614B9847044615B9337858
:1026A000012B0BD09CB95E4B1B6813F0010F0ED0B1
:1026B00000BE0CE008465B4B9847EAE700205A4B07
:1026C0009847EFE7544B1B7A13F0010F01D104B088
:1026D00070BD514B1A7A42F004021A725E6B11B946
:1026E0003378012B11D02146301D4C4B98470446BE
:1026F00015B93378012B0CD0002CE8D1484B1B685E
:1027000013F0010FE3D000BEE1E70020454B9847EE
:10271000E9E70020444B9847EEE73F4B1B7A13F064
:10272000010FD4D03C4A137A6FF382031372566BB5
:1027300011B93378012B11D02146301D374B984702
:10274000044615B93378012B0CD0002CBFD1344B83
:102750001B6813F0010FBAD000BEB8E70020314B60
:102760009847E9E70020304B9847EEE72A4B1B7A61
:1027700013F0040FABD0284A137A6FF3820313725D
:10278000002301930293039303788DF8043005230B
:102790008DF80530546B11B92378012B11D001A9A4
:1027A000201D1E4B9847064615B92378012B0CD0E7
:1027B000002E8CD11A4B1B6813F0010F87D000BE7E
:1027C00085E70020174B9847E9E70020164B98470C
:1027D000EEE7114B5E6B11B93378012B13D0214614
:1027E000301D0E4B9847044615B93378012B0ED097
:1027F000002C7FF46CAF0A4B1B6813F0010F3FF401
:1028000066AF00BE63E70020064B9847E7E700206D
:10281000054B9847ECE700BFEC0800208D214000F5
:10282000F0ED00E0713540006135400000B585B045
:1028300000230193029303938DF804008DF8051093
:10284000114601A8024B984705B05DF804FB00BF94
:102850005126400000B585B00023019302930393F5
:102860008DF8040001238DF805308DF8081011460D
:1028700001A8024B984705B05DF804FB51264000C3
:1028800000B585B0002301938DF8040006238DF870
:10289000053002AB0868496803C3114601A8024B22
:1028A000984705B05DF804FB5126400010B584B090
:1028B0000024019402948DF8040007208DF805008F
:1028C0008DF8081003928DF809309DF8181001A8B2
:1028D000014B984704B010BD5126400038B58B78A5
:1028E00003F07F03052B08D9104B1B6813F0010F71
:1028F00019D000BE0023184638BD0C4605460C4BC7
:10290000997A20460B4B9847034630B9074A12681C
:1029100012F0010FEFD000BEEDE721462846064B2E
:1029200098470346E7E70023E5E700BFF0ED00E046
:10293000EC080020ED3A4000F93540002DE9F04761
:1029400080460C4616461F46DDF82090DDF824A090
:10295000002513E0184B1B6813F0010F2AD000BEAE
:10296000002324E0144A126812F0010F1FD000BEA9
:102970001DE08AF8003023781C440135B54215DA91
:102980006378052BE6D1E37803F00303BB42E1D182
:1029900021464046094B984703460028E2D0A378D9
:1029A00013F0800FE5D189F80030E4E701231846E1
:1029B000BDE8F0870023FAE7F0ED00E0DD284000F5
:1029C00010B401F07F04C909124B03EB44030B441C
:1029D0002033DB7913F0010F0AD10E4A02EB4402D7
:1029E0000A4492F8273013F0040F10D0002200E0C0
:1029F000002210464AB1074B03EB4403194491F8F7
:102A0000273043F0040381F8273010BC70470122BF
:102A1000EFE700BFEC080020F8B501F07F06CD0914
:102A20001C4C04EB46042C442034E47914F0010FD0
:102A300008D0194B1B6813F0010F29D000BE0023EA
:102A40001846F8BD134C04EB46042C4494F8277048
:102A500047F0010784F82770104CA0470346002870
:102A6000EED10C4A02EB4606354495F827206FF369
:102A7000000285F8272095F827206FF3820285F859
:102A80002720054A126812F0010FD9D000BED7E7FF
:102A90000023D5E7EC080020F0ED00E0BD36400053
:102AA00038B501F07F05CC090E4B03EB45032344F9
:102AB0002033DB7913F0020F00D038BD0A4B984762
:102AC000084B03EB4503234493F8272042F002020E
:102AD00083F8272093F8272042F0010283F827206B
:102AE000EBE700BFEC0800206137400038B501F08B
:102AF0007F05CC090E4B03EB450323442033DB79E0
:102B000013F0020F00D138BD0A4B9847084B03EB76
:102B10004503234493F827206FF3410283F82720CD
:102B200093F827206FF3000283F82720EBE700BF1C
:102B3000EC0800209937400001F07F02044B03EBC2
:102B4000420303EBD11191F82700C0F34000704716
:102B5000EC0800202DE9F04182B005460C4600202B
:102B60009D4B98472378C3F34113022B0BDD9B4BFE
:102B70001B6813F0010F00F0D58100BE002318463A
:102B800002B0BDE8F081237803F06003402B12D03F
:102B9000227802F01F02012A00F0E880CAB1022A5E
:102BA00000F04E818D4B1B6813F0010F00F0D281B5
:102BB00000BE0023E3E78A4B002B00F0B5811E46E0
:102BC0001846854B9847224600212846B0470346C1
:102BD000D5E7202B0AD0002B30D0804B1B6813F098
:102BE000010F00F0A78100BE0023C8E7A388DBB275
:102BF0000F2B00F29B817B4A1344DB7A7A4AA2B105
:102C0000784A127993420ED203EB4303DA00754BF4
:102C100019681144002900F08B8122462846734B25
:102C200098470346ABE79B1ADBB22BB903EB430390
:102C3000DA006F491144EDE70021EBE76378092BD7
:102C400000F28B80DFE803F07464895489054E89B3
:102C500014202046674B98476188C9B22846664BC6
:102C60009847604A137A43F002031372012386E700
:102C70005C4B5B7A02AA02F8023D012321462846FA
:102C80005E4CA04701237AE76688F6B2554B5B7A23
:102C9000DBB29E4203D0534B5B7A43B99EB9514B92
:102CA0005E7221462846564B9847012367E728461F
:102CB000544B98474B4F97F80A802846524B9847F9
:102CC00087F80A80EAE731462846504B9847034682
:102CD0000028E4D1414A126812F0010F3FF44FAFCF
:102CE00000BE4CE721462846494B9847034646E735
:102CF0006388012B01D0002341E73A4A137A43F05D
:102D000008031372214628463D4B9847012336E7B6
:102D10006388012B01D0002331E7324B1A7A6FF31D
:102D2000C3021A7221462846354B9847012326E7ED
:102D30002C4B1B7AC3F3401213F0080F0BD1002366
:102D4000134302AA22F8023D0223214628462B4CB7
:102D5000A047012313E70223F2E7204B1B6813F07F
:102D6000010F00F0E98000BE002308E7A388DBB272
:102D70000F2B00F2E3801B4A1344DB7A1A4A002A25
:102D80004AD0184A1279934244D203EB4303DA0043
:102D9000144B19681144002900F0D28022462846BD
:102DA000124B9847034600287FF4E9AE227812F0D0
:102DB000600F7FF4E4AE62780A3A012A3FF6DFAE94
:102DC000054B984763780A2B2FD0214628460C4B99
:102DD00098470123D3E600BF29334000F0ED00E01F
:102DE00000000000EC08002000000000A9224000C4
:102DF000C83C4000353340004D3740007D32400034
:102E00003D324000B936400009224000C92240004E
:102E1000AD2440009B1ADBB22BB903EB4303DA006D
:102E20004D491144B7E70021B5E702AA002302F893
:102E3000023D012321462846484CA04701239EE637
:102E4000A288D1B201F07F06C2F3C012052E07D9C5
:102E5000434B1B6813F0010F74D000BE00238EE6B5
:102E6000404800EB46000244D27E3F48A8B13D48AE
:102E7000007982420FD202EB4202D000394A166832
:102E800006449BB1002E5FD0224631462846374B80
:102E90009847034673E6121AD2B22AB902EB4202ED
:102EA000D0002D4E0644ECE70026EAE76378012BBC
:102EB00017D04BB1032B14D0294B1B6813F0010F13
:102EC00046D000BE00235AE62846294B984702AA5E
:102ED00022F8020D022321462846204CA047012358
:102EE0004DE6628822B9012B18D02846214B98471D
:102EF00066B32246314628461C4B984700201E4B9D
:102F00009847184B93F8283013F001037FF437AE3D
:102F100021462846194B9847012330E62846184B8E
:102F20009847E5E700232AE6002328E6002326E663
:102F3000002324E6002322E6002320E600231EE6E9
:102F400000231CE600231AE6002318E6012316E6F8
:102F5000002314E6002312E6C83C40007D32400006
:102F6000F0ED00E0EC08002000000000A922400085
:102F7000392B4000A12A4000293340003D32400057
:102F8000ED2A400030B585B0884B984788B905B028
:102F900030BD0020864B984710E00020854B9847B5
:102FA00014E09DF80400844B98479DF80820834B5B
:102FB0009A72824B5C6B2378012BEAD001A9201D09
:102FC0007F4B984705462378012BE6D0002DDED0B5
:102FD0009DF80530013B072B00F2E08001A252F87A
:102FE00023F000BFA32F4000053040008B3140008C
:102FF000093140002B314000173040007330400051
:103000008F3140009DF804006B4B98476D4B002BAF
:10301000CFD09847CDE7694B1A7A42F001021A7275
:1030200093F827206FF3000283F8272093F82720D6
:103030006FF3820283F8272093F828206FF30002B1
:1030400083F8282093F828206FF3820283F8282041
:1030500002A99DF804005C4B98470028A9D10021E3
:103060009DF80400594CA04780219DF80400A0471A
:103070009FE79DF8081001F07F00CC094F4B03EB50
:103080004003234493F827206FF3000283F827209E
:1030900093F827206FF3820283F8272088B1474BEB
:1030A00003EB40032344DB7E494AA2B1434A127931
:1030B00093420ED203EB4303DA00404B1B681344E8
:1030C0000FE0039B9DF809209DF80400414CA047A8
:1030D0006FE79B1ADBB26BB903EB4303DA003E4B9D
:1030E00013444BB11C69039B9DF809209DF8040013
:1030F000A0475EE70023F4E7384B1B6813F0010F8D
:103100003FF445AF00BE42E72C4B1B7A13F0010F92
:103110003FF44FAF324B002B3FF44BAF274B187AA5
:10312000C0F3C0002E4B984743E7244B1B7A13F0A3
:10313000010F3FF43EAF2B4B002B3FF43AAF9847C3
:1031400037E7E31ADBB2F3B903EB4303DA00224BB0
:1031500013445B6913B19DF8040098470134E4B24D
:10316000164B1B795A1C9442BFF623AF184A42B142
:103170009C42E6D204EB4403DA00104B1B68134474
:10318000E7E72346DFE70023E3E70024E8E7029BC5
:10319000002B3FF40EAF039898470AE70F4B1B68CC
:1031A00013F0010F3FF405AF00BE02E7DD3A400027
:1031B000713540006135400095224000EC08002048
:1031C0006121400000000000552B400061374000A5
:1031D0000000000055334000C83C4000F0ED00E026
:1031E000000000000000000038B50546104BB3F8A1
:1031F0004C40B3F84E20A41AA4B2402C28BF40245F
:1032000093F94030002B07DB00217CB900222346D4
:103210002846084CA04738BD0CB98021F5E7044882
:103220002246816C044B98478021EEE7004AEEE786
:1032300024090020192A4000893C400038B5054681
:103240000C460C4B03F140020868496803C2002297
:103250009A64A3F84E20A3F84C2094F900309342CE
:1032600006DB802100231A462846034CA04738BDC0
:103270001146F7E724090020192A4000F8B507464F
:103280000C46204D05F140060868496803C6AA644B
:103290000021A5F84E10E1888B4228BF0B46A5F807
:1032A0004C30E188A9B103B15AB13846164B984762
:1032B000034600BB154A126812F0010F1BD000BE76
:1032C00019E0124B1B6813F0010F18D000BE002349
:1032D00011E094F90030002B0FDB802100231A4607
:1032E00038460B4CA047034628B9084A126812F02A
:1032F000010F00D000BE1846F8BD0021EEE7002304
:10330000F9E700BF24090020E9314000F0ED00E0BA
:10331000192A4000034900230B644B648B64CB647F
:103320000B65704724090020014B1865704700BFEA
:10333000240900200146064B03F140020068496859
:1033400003C200229A64A3F84E20A3F84C207047D1
:103350002409002038B505461C463C4B93F8403004
:10336000DB09B3EBD11F17D03CB1394B1B6813F00D
:10337000010F65D000BE00230CE0364B0BB136497F
:103380009847324B1B6D002B5CD0334A02212846F4
:1033900098470123184638BD2C4B93F94030002B39
:1033A00007DB2A4B986C00284ED0224619462B4B3F
:1033B0009847264AB2F84E3023449BB2A2F84E30CA
:1033C000916C21449164B2F84620934201D03F2C85
:1033D00029D81E4B1B6DCBB11F4A012128469847A7
:1033E000C0B11A4B93F94030002B11DB8021002330
:1033F0001A4628461A4CA04703460028CAD1144A48
:10340000126812F0010FC5D000BEC3E70120E7E744
:103410000021ECE700212846124CA04780212846D5
:10342000A0470123B6E728460F4B984703460028DC
:10343000B0D1074A126812F0010FABD000BEA9E765
:103440000023A7E70123A5E70023A3E72409002021
:10345000F0ED00E0BD35400064090020893C4000EB
:10346000192A400061374000E931400000239342AF
:103470000CD270B4CE5C00F11404054D45F8246004
:1034800001339BB29342F5D370BC7047704700BFC5
:1034900000400440002393420CD230B400F11404E5
:1034A000054D55F82440CC5401339BB29342F5D3DB
:1034B00030BC7047704700BF004004400181704736
:1034C00010B582B0104C4822002120460F4B98477F
:1034D000402120460E4B98474FF400420D4B1A6393
:1034E0000023019303E000BF019B01330193019B83
:1034F000132BF8D9074B42F201321A615A6F22F4AA
:1035000080725A6702B010BDEC0A00209F3C400058
:10351000BD34400000400440016082800023C3802D
:103520007047002303608380C38070478388C2880C
:1035300092B29B1A9BB20089984228BF18467047E6
:1035400010B50446054B9847236803442360E3887D
:1035500010FA83F080B2E08010BD00BF2D3540002E
:103560004FF48032014B5A60704700BF00E100E029
:103570004FF48032034BC3F88420BFF34F8FBFF367
:103580006F8F704700E100E04FF44072014B5A67C3
:10359000704700BF0040044010B504464822002197
:1035A0000348044B98472046034B984710BD00BF83
:1035B000EC0A00209F3C4000893540000B7813F056
:1035C0007F0F04D14B78052B02D0092B0CD070470C
:1035D0004B88084A516841F00101516003F07F03B4
:1035E00043F4807393607047024A536843F00203C8
:1035F0005360ECE700400440F0B583B08C78CB78A2
:1036000003F00303012B48D004F07F0564B2E70FF9
:10361000052D44D805F10C03234A52F8233013F446
:10362000004F07D0214B1B6813F0010F3AD000BEAA
:10363000002035E00E460979737903F0070305EBA6
:103640004500820041EA032119481044194B98476C
:10365000F37803F0030303EB87031B0203F4E06337
:1036600043F4004305F10C020F4941F822300023D6
:10367000019303E000BF019B01330193019B132BD6
:10368000F8D9002C01DB01200AE0074A1369012068
:1036900000FA05F51D43156102E0002000E000205E
:1036A00003B0F0BD0020FBE700400440F0ED00E077
:1036B000EC0A0020BD34400070470000F0B583B034
:1036C000174601F07F044DB204EB440082001A4E0D
:1036D00016441A4639463046184B9847002D0ADBE7
:1036E00034B117490B69012202FA04F41C430C613E
:1036F000012003B0F0BD04EB440293000E4AD558FC
:103700003046104B98470246294620460E4B9847B4
:103710000B4A0C3452F8243043F05F0342F8243053
:103720000023019303E000BF019B01330193019B40
:10373000132BF8D9DCE700BFEC0A00201935400054
:10374000004004402D3540006D34400010B500238A
:103750001A468021014CA04710BD00BFBD36400075
:10376000802915D082B001F07F010A4A0C3152F84D
:10377000213043F06F0342F821300023019303E02E
:1037800000BF019B01330193019B132BF8D902B0B9
:10379000704700BF0040044082B001F07F01114A31
:1037A00001F10C0052F8203023F0200343F04F03C6
:1037B00042F820300023019303E000BF019B013356
:1037C0000193019B132BF8D9064B986A012202FA48
:1037D00001F1084398629A6A22EA0101996202B0F3
:1037E000704700BF004004402DE9F0478AB006460C
:1037F000A54B9D69DA6915401D6215F4805F12D1F1
:1038000015F4807F17D115F4007F1AD115F4005FED
:103810001DD115F0010F04D09B4B1B6B13F0040F4F
:1038200038D10024F9E0994B984701220021304615
:10383000974B9847E4E7012204213046954B98477F
:10384000E1E7012205213046924B9847DEE701224D
:10385000052130468F4B9847DBE78B4A116D0AAA4A
:103860001A4402F8081C0133DBB2072BF5D90122F8
:1038700008A93046884B98479DF92030002B0BDB78
:10388000814A136B23F0800343F04F03136300233B
:10389000039315E00023E8E77B4A136B43F0CF0363
:1038A00013630023029303E000BF029B01330293E2
:1038B000029B132BF8D906E000BF039B013303934F
:1038C000039B132BF8D9704A136B23F07F03136308
:1038D0000023049303E000BF049B01330493049B83
:1038E000132BF8D99DE740466C4B984740466C4BEC
:1038F0009847024640B304EB44018B006949C9581C
:103900002046694B9847604A04F10C0152F8213077
:1039100043F05F0342F821300023059303E000BF2A
:10392000059B01330593059B132BF8D9564A07F1E4
:103930000C0152F8213023F0010343F04E0342F80A
:1039400021300023069317E004EB44039A00554B03
:103950001344DA8801230093002392B244F08001DB
:103960003046DFF85091C8474046504B9847DDE756
:1039700000BF069B01330693069B132BF8D963E027
:1039800007F10C0352F8232007EB47018B00C2F329
:103990000A424449C9582046454B984740463F4B48
:1039A000984740463E4B9847C0B92CB136494B69C1
:1039B0000122BA4013434B6107EB47039A00394B8E
:1039C0001344DA8801230093002392B22146304643
:1039D000DFF8E0A0D0474046344B98472A4A07F129
:1039E0000C0152F8213043F04F0323EA090342F857
:1039F00021300023079303E000BF079B01330793A7
:103A0000079B132BF8D927E000BF089B01330893CD
:103A1000089B132BF8D90134E4B2052C30D8274683
:103A200025FA04F313F0010FF5D004EB44034FEA39
:103A300083081C4B984404F10C03134A52F82330BA
:103A400013F0010F7FF44FAF07F10C030E4A52F849
:103A5000233013F0420993D107F10C030A4A52F8BC
:103A6000233013F0080FD6D00C3752F8273023F04C
:103A7000080343F0470342F8273000230893C7E7C1
:103A80000AB0BDE8F08700BF00400440C1344000E8
:103A9000552840002D284000812840004135400035
:103AA0002D354000EC0A00206D34400023354000E5
:103AB00095344000AD28400008B50020054B9847DC
:103AC000034628B9044A126812F0010F00D000BE64
:103AD000184608BDA1254000F0ED00E008B5024BF6
:103AE000984700B1012008BD95254000027943792F
:103AF00003F0070342EA0322C37803F00303022B17
:103B000013D029D8012B37D102290BD040F2FF3333
:103B1000934233D2214B1B6813F0010F30D000BE0B
:103B2000002070474FF48063F2E7022909D0402A51
:103B30002CD91A4B1B6813F0010F29D000BE0020AE
:103B40007047B2F5007F1DD0144B1B6813F0010FB6
:103B50001AD000BE0020704702290AD040239342A9
:103B600018D20E4B1B6813F0010F15D000BE0020B9
:103B700070474FF48063F2E70020704701207047E0
:103B800000207047012070470020704701207047D7
:103B9000002070470120704700207047F0ED00E0E2
:103BA00070B4002403E00D782C44A4B2294494425C
:103BB0000AD24D78052DF6D18D7805F07F0600EB01
:103BC0004606ED097355EEE770BC70470048704734
:103BD000E03C400000487047F43C4000004870471B
:103BE000183D400010B560B9124B1B681A88124B83
:103BF0005A800120431C5B0043F440730E4803804D
:103C000010BD032814D80B4A52F8204020460B4B15
:103C10009847C0B21F2800D91F20002305E05A1C76
:103C2000E15C054B23F81210D3B29842F7D8E1E7D4
:103C3000002010BDF401002078090020AF3C4000B6
:103C400070B50D4E0D4CA41BA4100025A54209D142
:103C50000B4E0C4C00F092F8A41BA4100025A542BA
:103C600005D170BD56F8253098470135EEE756F876
:103C7000253098470135F2E7883D4000883D4000F7
:103C8000883D40008C3D400010B5431E0A449142DF
:103C900000D110BD11F8014B03F8014FF7E70244C2
:103CA0000346934200D1704703F8011BF9E703462E
:103CB00013F8012B002AFBD1181A013870470000B5
:103CC000302E322E31000000691C4000511C400093
:103CD000791C4000951D40001920400000000000A4
:103CE0001201000200000040BD3504400001010245
:103CF000030100000600FF0901A1010902150026C9
:103D0000FF007508954081020903150026FF007524
:103D10000895409102C000000902290001010080BD
:103D20003209040000020300000009211101000112
:103D30002222000705020340000A07058103400014
:103D40000A00000009040000426967736372656538
:103D50006E00000042696773637265656E2055539B
:103D600042204669726D7761726520557067726195
:103D7000646500003132333435360000F8B500BFD9
:103D8000F8BC08BC9E46704729044000F8B500BF47
:103D9000F8BC08BC9E4670470504400082B0154B35
:103DA0001A6842F480321A60134A5A60114B9B68B9
:103DB0000193019B13F0010FF8D1002306E09A0054
:103DC00002F58002126840F8232001338B42F6D3BB
:103DD0000A4A084B5A60074B9B680193019B13F0FA
:103DE000010FF8D0034A136823F48033136002B044
:103DF000704700BF000A0E400E00005A0F00005A24
:103E000082B00F4B58600E4B9B680193019B13F0DF
:103E1000010FF8D0019B13F0020F02D0022002B074
:103E20007047019B13F0080F01D00320F7E7019BB7
:103E300013F0040F01D10020F1E70120EFE700BFEC
:103E4000000A0E4082B0104B58600F4B9B680193E4
:103E5000019B13F0010FF8D0019B13F0020F02D069
:103E6000022002B07047019B13F0080F01D003201D
:103E7000F7E7019B13F0040F04D1034BDB680B60E1
:103E80000020EEE70120ECE7000A0E4010B483B0FA
:103E9000214C6060204880680190019810F0010F6B
:103EA000F8D1019810F0020F03D0022003B010BC2B
:103EB0007047019810F0080F01D00320F6E7019831
:103EC00010F0040F26D1002005E0144C54F82040D7
:103ED00042F8204001309842F7D30F4B59600E4B07
:103EE0009B680193019B13F0010FF8D0019B13F025
:103EF000020F01D00220D9E7019B13F0080F01D077
:103F00000320D3E7019B13F0040F01D10020CDE77C
:103F10000120CBE70120C9E7000A0E400000400065
:103F200000127A000100000040000000887B0020A1
:103F300019114100151141001511410015114100E1
:103F400015114100151141000000000000000000A3
:103F50000000000000000000B114410015114100F4
:103F6000000000001115410075154100010000001E
:103F70002C0A002010000C000000E0FF1F000000D1
:103F800000000000443D4000483D4000543D4000DA
:103F9000743D4000FFFFFFFFFFFFFFFF1C8D408AC5
:00000001FF
